:100000000C949C060C94D4060C94D4060C94D40640
:100010000C94D4060C94D4060C94D4060C94D406F8
:100020000C94D4060C94D4060C94D4060C944E2B49
:100030000C94FD2B0C94F9250C94D4060C94D40646
:100040000C94D4060C94D4060C94D4060C948126FB
:100050000C94D4060C94D4060C94D4060C94D406B8
:100060000C94D4060C94D4060C94D4060C94D406A8
:100070000C94D4066B0A6B0A970A970A0C0C0C0CAA
:100080000C0C0C0CFF0A980BA90BA90B41222F2278
:100090004822BA21F522F5222C22F522F5227522DA
:1000A000F5228922D522F522F522F522F522A92270
:1000B000F522F522A622F5226122F522F522EF2271
:1000C000EF22EF22EF22EF22EF22EF22EF22EF22A8
:1000D000F122F52241222422F522F522F522F522F1
:1000E000F522F522F522F522F522F522F122F5225C
:1000F000F5222C22F522ED22ED22ED22ED22ED2239
:10010000ED22ED22ED22ED22F1226A2C912C892D97
:10011000912C892DDD2C002D892D572D662D4A001F
:100120004D0044454255473A2064697361626C65ED
:10013000642E0A0044454255473A20656E61626C60
:1001400065642E0A000A0025303258006C65645F31
:100150007461736B3A20004F6E6573686F743A2058
:100160006163746976653A2025640A000A002530C7
:100170003862003A200025303258000A722F63207E
:1001800030313233343536370A007267626C696752
:1001900068742074696D65722064697361626C654E
:1001A0002E0A007267626C696768742074696D65F5
:1001B0007220656E61626C65642E0A007267626C03
:1001C000696768742073657420687376205B4E4F8E
:1001D000454550524F4D5D3A2025752C25752C25EF
:1001E000750A007267626C696768742073657420B1
:1001F000687376205B454550524F4D5D3A2025751A
:100200002C25752C25750A007267626C6967687405
:10021000207261696E626F772073657420687376EF
:100220003A2025642C25642C25642C25750A00723F
:1002300067626C696768742064697361626C6520C9
:100240005B454550524F4D5D3A207267626C69675D
:1002500068745F636F6E6669672E656E61626C6558
:10026000203D2025750A007267626C6967687420FA
:10027000656E61626C65205B454550524F4D5D3A3D
:10028000207267626C696768745F636F6E66696726
:100290002E656E61626C65203D2025750A007267CF
:1002A000626C6967687420746F67676C65205B4572
:1002B0004550524F4D5D3A207267626C69676874B1
:1002C0005F636F6E6669672E656E61626C65203D67
:1002D0002025750A007267626C69676874206D6F0B
:1002E0006465205B4E4F454550524F4D5D3A202589
:1002F000750A007267626C69676874206D6F646567
:10030000205B454550524F4D5D3A2025750A0072DD
:1003100067626C696768745F696E6974207267628E
:100320006C696768745F636F6E6669672E6D6F6472
:1003300065203D20302E2057726974652064656603
:1003400061756C742076616C75657320746F2045DF
:100350004550524F4D2E0A007267626C696768748F
:100360005F696E6974206565636F6E666967206991
:1003700073206E6F7420656E61626C65642E0A0076
:100380007267626C696768745F696E697420737400
:10039000617274210A007267626C696768745F69D0
:1003A0006E69742063616C6C65642E0A007267620A
:1003B0006C696768745F636F6E6669672E737065DA
:1003C0006564203D2025640A007267626C69676875
:1003D000745F636F6E6669672E76616C203D2025C1
:1003E000640A007267626C696768745F636F6E6647
:1003F00069672E736174203D2025640A007267626C
:100400006C696768745F636F6E6669672E6875658F
:10041000203D2025640A007267686C696768745F14
:10042000636F6E6669672E6D6F6465203D2025647D
:100430000A007267626C696768745F636F6E6669F1
:10044000672E656E61626C65203D2025640A00722E
:1004500067626C696768745F636F6E666967204581
:100460004550524F4D3A0A0000047F3F1F6432143A
:10047000643214783C1E1E140A05222325262829DE
:100480002A2C2D2F3032333536383A3B3D3E404210
:10049000434547494A4C4E5051535557595A5C5E53
:1004A0006062646668696B6D6F71737577797B7D67
:1004B0007F81838587898A8C8E90929496989A9C66
:1004C0009E9FA1A3A5A7A8AAACAEAFB1B3B4B6B87E
:1004D000B9BBBCBEBFC1C2C3C5C6C7C9CACBCCCDE0
:1004E000CED0D1D2D2D3D4D5D6D7D7D8D9D9DADABB
:1004F000DBDBDBDCDCDCDCDCDDDDDDDDDCDCDCDC3B
:10050000DCDBDBDBDADAD9D9D8D7D7D6D5D4D3D26E
:10051000D2D1D0CECDCCCBCAC9C7C6C5C3C2C1BF4C
:10052000BEBCBBB9B8B6B4B3B1AFAEACAAA8A7A5B0
:10053000A3A19F9E9C9A98969492908E8C8A89876C
:100540008583817F7D7B79777573716F6D6B69684A
:10055000666462605E5C5A5957555351504E4C4A1E
:100560004947454342403E3D3B3A383635333230C9
:100570002F2D2C2A292826252322FFAA7F5540002B
:100580000101010101010101010202020202020254
:100590000202030303030303030304040404040427
:1005A00004050505050506060606060707070707ED
:1005B00008080808090909090A0A0A0B0B0B0C0CA0
:1005C0000C0D0D0D0E0E0E0F0F0F1010111111123C
:1005D0001213131414151516161717181819191ABB
:1005E0001A1B1B1C1D1D1E1E1F202021222223241E
:1005F00024252626272829292A2B2C2D2D2E2F305D
:10060000313232333435363738393A3B3C3D3E3F70
:10061000404142434445464748494A4C4D4E4F505D
:10062000515354555658595A5B5D5E5F616264651B
:100630006668696B6C6D6F7072737577787A7B7DA5
:100640007E8082838587888A8C8E8F9193959698F9
:100650009A9C9EA0A2A3A5A7A9ABADAFB1B3B5B715
:10066000BABCBEC0C2C4C6C9CBCDCFD1D4D6D8DBEC
:10067000DDDFE2E4E7E9EBEEF0F3F5F8FAFDFF3F4A
:1006800000433E20004C25640A000A092D205374C3
:1006900061747573202D0A686F73745F6B6579627E
:1006A0006F6172645F6C65647328293A202530326B
:1006B000580A6B6579626F6172645F70726F746FF4
:1006C000636F6C3A20253032580A6B6579626F612E
:1006D00072645F69646C653A20253032580A6B6534
:1006E000796D61705F636F6E6669672E6E6B726F96
:1006F0003A20253032580A74696D65725F726561FF
:1007000064333228293A202530386C580A000A0907
:100710002D2056657273696F6E202D0A5649443A32
:1007200020307846454544284B696E676C792D4BDF
:1007300065797329205049443A203078423139355F
:1007400028534D442D3225204D696C6B2920564588
:10075000523A203078303030310A4255494C443AD0
:100760002020284665622032372032303232290A72
:100770004F5054494F4E533A204C55464120434F19
:100780004E534F4C4520434F4D4D414E44204E4B10
:10079000524F20343039360A4743433A20352E34FD
:1007A0002E30204156522D4C4942433A20322E30B1
:1007B0002E30204156525F415243483A20617672B2
:1007C00033350A000A092D20436F6E736F6C652064
:1007D0002D0A4553432F713A09717569740A000A4D
:1007E000092D204D61676963202D0A443A0944654B
:1007F000627567204D65737361676520546F676725
:100800006C650A583A094D617472697820446562D2
:100810007567204D6F646520546F67676C65202D88
:100820002053686F77206B65797072657373657399
:1008300020696E206D617472697820677269640A3C
:100840004B3A094B6579626F617264204465627549
:100850006720546F67676C65202D2053686F772081
:100860006B65797072657373207265706F72740A4C
:100870004D3A094465627567204D6F757365205464
:100880006F67676C650A563A0956657273696F6ED1
:100890000A533A095374617475730A433A09416300
:1008A00074697661746520436F6E736F6C65204D5B
:1008B0006F64650A46312D4631303A0953776974C1
:1008C000636820746F204C6179657220302D392067
:1008D00028463130203D204C30290A302D393A0944
:1008E00053776974636820746F204C617965722056
:1008F000302D390A47524156453A09537769746396
:100900006820746F204C6179657220302028616CFA
:100910007465726E617465290A423A094A756D7090
:1009200020746F20426F6F746C6F616465720A454A
:1009300053433A094A756D7020746F20426F6F748B
:100940006C6F616465722028616C7465726E61748D
:1009500065290A453A095072696E7420454550521E
:100960004F4D2053657474696E67730A425350414A
:1009700043453A09436C65617220454550524F4DDD
:100980000A4E3A094E4B524F20546F67676C650A06
:10099000006B65796D61705F636F6E6669672E725B
:1009A00061773A20253032580A2E737761705F6381
:1009B0006F6E74726F6C5F636170736C6F636B3AB0
:1009C0002025750A2E636170736C6F636B5F746FA3
:1009D0005F636F6E74726F6C3A2025750A2E7377A1
:1009E00061705F6C63746C5F6C6775693A20257524
:1009F0000A2E737761705F7263746C5F72677569DA
:100A00003A2025750A2E737761705F6C616C745F94
:100A10006C6775693A2025750A2E737761705F726D
:100A2000616C745F726775693A2025750A2E6E6F66
:100A30005F6775693A2025750A2E737761705F6765
:100A4000726176655F6573633A2025750A2E737748
:100A500061705F6261636B736C6173685F62616335
:100A60006B73706163653A2025750A2E6E6B726F29
:100A70003A2025750A0064656275675F636F6E666C
:100A800069672E7261773A20253032580A2E656EDA
:100A900061626C653A2025750A2E6D617472697801
:100AA0003A2025750A2E6B6579626F6172643A206F
:100AB00025750A2E6D6F7573653A2025750A0065D8
:100AC00065636F6E6669673A0A64656661756C7422
:100AD0005F6C617965723A2025750A003F004E4BC4
:100AE000524F3A206F66660A004E4B524F3A206FC3
:100AF0006E0A000A6D6F7573653A206F66660A00AC
:100B00000A6D6F7573653A206F6E0A000A6B65791E
:100B1000626F6172643A206F66660A000A6B6579DB
:100B2000626F6172643A206F6E0A000A6D617472BE
:100B300069783A206F66660A000A6D617472697896
:100B40003A206F6E0A000A64656275673A206F6624
:100B5000660A000A64656275673A206F6E0A000AC9
:100B60000A4A756D70696E6720746F20626F6F74CA
:100B70006C6F616465722E2E2E2000433E20004370
:100B80006C656172696E6720454550524F4D0A0091
:100B90000A002530325820006B6579626F617264FB
:100BA0005F7265706F72743A200064656C5F6B658C
:100BB000795F6269743A2063616E27742064656CA2
:100BC0003A20253032580A006164645F6B65795FB2
:100BD0006269743A2063616E2774206164643A200C
:100BE000253032580A005B735D005B575D005B5334
:100BF0005D005B525D00180353004D0044002D0062
:100C00003200250020004D0069006C006B000000E0
:100C100018034B0069006E0067006C0079002D001E
:100C20004B00650079007300000004030904090209
:100C30005B00030100A0FA090400000103010100A8
:100C4000092111010001224000070581030800016C
:100C50000904010001030000000921110100012223
:100C60003B00070582032000010904020002030083
:100C70000000092111010001222200070583032041
:100C8000000107050303200001120100020000001B
:100C900008EDFE95B10100010200010631FF097463
:100CA000A1010975150026FF00952075088102092C
:100CB00076150026FF00952075089102C0050109F0
:100CC00006A1018506050719E029E715002501950C
:100CD00008750181020507190029EF150025019506
:100CE000F075018102050819012905950575019125
:100CF00002950175039101C005010906A1010507CF
:100D000019E029E715002501950875018102950173
:100D1000750881010507190029FF150026FF0095B8
:100D200006750881000508190129059505750191C9
:100D300002950175039101C011241FBECFEFD4E0CD
:100D4000DEBFCDBF04B603FE18C080915B02909158
:100D50005C02A0915D02B0915E028730904BA7408B
:100D6000B04B59F410925B0210925C0210925D023B
:100D700010925E02E0E0F8E3099511E0A0E0B1E036
:100D8000EEE5FDE502C005900D92AA35B107D9F751
:100D900022E0AAE5B1E001C01D92AB35B207E1F750
:100DA0000E948D170C94AD2E0C940000FF93EF93CE
:100DB000E0915A01F0915B01309709F00995EF91AC
:100DC000FF910895FC018591803011F0EFDFFBCF9A
:100DD0000895FF27E0E230E247FF0CC0419597FFFE
:100DE00009C0EDE26095709580959095611D711D2B
:100DF000811D911D27FF02C0219530E350E2AA27F3
:100E0000660F771F881F991FAA1FA41710F0A41B35
:100E100063955A95A9F7AA3008F0A95FA05DAF9332
:100E2000F395611571058105910541F7ED3211F4D6
:100E3000EF93F395F21718F43F93F395FBCF8F914F
:100E4000B5DFFA95E1F70895E991F9918591803040
:100E500021F0853219F0AADFF9CF089520E0E89457
:100E600055915532C1F3503311F4689455915A336A
:100E700048F4505390F3220F022E220F220F200D20
:100E8000250FF4CF0EF4219589919991533619F3DA
:100E9000533729F1533559F1BC0188279927E89434
:100EA0005C3621F48991999168945591543639F4BE
:100EB00046EF7EF077FF0DC08FEF9FEF0AC05537EA
:100EC0004AE039F0583540E121F0523642E009F06D
:100ED0000895FF93EF937DDFEF91FF91B7CFFF93DD
:100EE000EF93FC0181918030B9F360DFFBCFFF937A
:100EF000EF9368DFF1CFDF93CF93CDB7DEB72596C1
:100F0000A3DFCF91DF91089581E0089581E00895F6
:100F10000C94860708950C948A071F93CF93DF9350
:100F200000D000D01F92CDB7DEB749835A836B83C0
:100F300030915D0189819A81311114C0662359F085
:100F4000222349F00E943C0E182F682F89819A8134
:100F50000E94E60D03C00E94120E182F69817A814B
:100F6000812F04C00E943C0E69817A810F900F90FE
:100F70000F900F900F90DF91CF911F910C94371528
:100F8000FC01262F408151816281738184810C9400
:100F90008D0781E00895CF93DF93EC0160E00E941C
:100FA000C007BE01DF91CF910C948B070C94A31660
:100FB0000C949F1608950E94900C0E94DA072FEF60
:100FC00084E39CE0215080409040E1F700C00000A5
:100FD0000C94A7260F931F93CF93DF938C0161E0AE
:100FE0000E94C007EC01B8010E948807882309F419
:100FF00062C0B801CE010E94F423882309F45BC0CB
:10100000B801CE010E943F20882309F454C0B801E2
:10101000CE010E945023882309F44DC0B801CE01AF
:101020000E94451F882309F446C0F8018281882365
:10103000D9F1CF3D8CE5D80779F140F4C115FCE535
:10104000DF0791F0C130DC4591F02EC0CC35EDE5E5
:10105000DE0741F1CD35FDE5DF0709F1CB35DD4593
:1010600019F50E94CF1220C00E94DB0724C0809196
:10107000F101C82FC095C170C0FB80F98093F101C8
:10108000CC2329F084E391E00E94E20614C082E2BE
:1010900091E00E94E20610C00E947D130CC00E94E5
:1010A000C61202C00E94D212C801DF91CF911F91D7
:1010B0000F910C948407C0E08C2FDF91CF911F918A
:1010C0000F9108950E94DA250C948D080E949008D3
:1010D0000C94E0258295982F9373292F220F220FCD
:1010E000982F9C7C96959695922B892F8575880FC5
:1010F0009A7A9695892B089508950C947C0881E03E
:1011000008950C947F080895CF93C82F0E947D08FE
:101110008C2F0E948108CF91089580E00C94840860
:101120000E9450240C948408CF930E945024C82F0E
:1011300080915C01C81741F1C0935C018091F1017D
:1011400082FF1EC080FF04C08CE491E00E94E20692
:101150008091F10180FF0CC01F92CF9387E491E052
:101160009F938F930E947B070F900F900F900F908B
:101170008091F10180FF04C085E491E00E94E206C5
:101180008C2FCF910C948408CF910895CF93DF9347
:10119000CDB7DEB72B970FB6F894DEBF0FBECDBF2D
:1011A0004F83588769877A878B8761110E94FE1168
:1011B0009E012F5F3F4F86E0F90111928A95E9F772
:1011C00085E0FE013796D90101900D928A95E1F7ED
:1011D00089819A814C815D81452B31F09F3F31F4AB
:1011E00091E08F3F19F403C091E001C090E090FFBF
:1011F00009C049815A816B817C818D819E810E94C9
:101200001A1105C0C9010E94C9078111F2CF2B969E
:101210000FB6F894DEBF0FBECDBFDF91CF9108951A
:10122000FC01808191810E947E0E0895CF938823D6
:1012300009F487C0C82F8238C1F40E94502481FD70
:1012400080C069E380910201909103010E9495257D
:101250000E9420122FEF81EE94E0215080409040B8
:10126000E1F700C0000069E319C08338F1F40E947F
:10127000502480FD66C063E58091020190910301D6
:101280000E9495250E9420122FEF81EE94E02150BC
:1012900080409040E1F700C0000063E580910201CA
:1012A000909103010E94A02549C08438C1F40E9496
:1012B000502482FD46C067E48091020190910301B1
:1012C0000E9495250E9420122FEF81EE94E021507C
:1012D00080409040E1F700C0000067E4DFCF8CEF72
:1012E0008C0F813AF8F48C2F0E940723811129C0BA
:1012F0006C2F80910201909103010E94F3248823B6
:1013000049F06C2F80910201909103010E94A02569
:101310000E9420126C2F80910201909103010E9483
:1013200095250CC080E28C0F883058F4C77081E09E
:1013300001C0880FCA95EAF70E94E111CF910C9481
:101340002012CF910895882309F45BC0682F82385A
:1013500079F40E94502481FF54C069E38091020116
:10136000909103010E9495250E94201269E310C00C
:101370008338B1F40E94502480FF43C063E580911C
:101380000201909103010E9495250E94201263E5BD
:1013900080910201909103010E94A0250C942012DB
:1013A000843879F40E94502482FF2BC067E4809136
:1013B0000201909103010E9495250E94201267E48A
:1013C000E7CF8CEF860F813A18F380E2860F8830E2
:1013D00048F4677081E001C0880F6A95EAF70E94BF
:1013E000E711DCCF8BE5860F833020F480E090E0BE
:1013F0000C94B124685A673120F480E090E00C949A
:10140000C72408951F93CF93DF93182FEB010E94F9
:101410001609209741F08FE99FE00197F1F700C08E
:1014200000002197F6CF812FDF91CF911F910C946F
:10143000A309893319F060E070E002C060E570E054
:101440000C94020A882321F00E94E1110C942012CE
:101450000895882321F00E94E7110C94201208952A
:10146000CF92DF92EF92FF920F931F93CF93DF9370
:101470007C01D62FC72FFC011281058102950F70C8
:101480000E94D7118823B9F01123A9F08C2F807FF7
:10149000803421F080E28D0F883068F08091340232
:1014A00082FD09C082E00E9480120E94D71191E063
:1014B000D82ED92601C0D12CCC2EC2948FE0C822C0
:1014C0008C2D90E08C30910508F0A6C1FC01E65C03
:1014D000FF4F0C94452E8C2F807FCF70882311F006
:1014E000C295C07F112399F0CC2309F481C180E219
:1014F0008D0F883010F0D11104C08C2F0E94E111A3
:1015000003C08C2F0E94F1110E94201271C18D2FF7
:101510000E94A309CC2309F47FC180E28D0F88309B
:1015200038F1DD2329F18C2F0E94F71124C08C2F74
:10153000807FCF70803211F0C295C07FDD2319F01B
:10154000D130A1F13DC08091340282FF17C0112338
:1015500049F0CC2329F08C2F0E94E1110E94201227
:1015600080E047C180E00E94A309CC2309F454C164
:101570008C2F0E94E7110E9420124EC1112371F09E
:10158000002341F0013031F40E9401128C2B0E94A3
:10159000091242C10E9401128C2B1DC0002319F0B8
:1015A000013009F439C10E94161225C0112321F01F
:1015B000063008F031C10EC0053008F02DC11BC047
:1015C000112361F0002331F0F701858180FF10C104
:1015D0008F7085838C2F0E94220A1EC1002359F030
:1015E000D93309F016C1FFEF07EE13E0F1500040C8
:1015F0001040E1F70CC18C2F0E94290A0DC18C2FDD
:10160000837009F047C011110BC12D2F229526952B
:101610002770220F220F6D2F6F70862F90E0A0E0B1
:10162000B0E0022E04C0880F991FAA1FBB1F0A94A6
:10163000D2F7D4FF10C04FE050E060E070E004C08B
:10164000440F551F661F771F2A95D2F74095509576
:101650006095709503C040E050E0BA01C695C6950C
:10166000C3708A019B01082B192B2A2B3B2BC90124
:10167000B801C23049F058F4C13019F00E94FC0C96
:10168000CFC00E94EA0CCCC00E940E0DC9C00E94BF
:10169000E80CC6C0112319F08C2F817001C086950B
:1016A000882309F4BDC02D2F229526952770220F7F
:1016B000220F6D2F6F70862F90E0A0E0B0E0022E19
:1016C00004C0880F991FAA1FBB1F0A94D2F7D4FF2A
:1016D00010C04FE050E060E070E004C0440F551FC0
:1016E000661F771F2A95D2F74095509560957095A3
:1016F00003C040E050E0BA01C695C695C3708A01A8
:101700009B01082B192B2A2B3B2BC901B801C23096
:1017100049F058F4C13019F00E94C10D81C00E94F7
:10172000AF0D7EC00E94D30D7BC00E94220D78C0F9
:10173000CF70112339F08C2F0E94480D8D2F0E94FD
:10174000220A6EC08D2F0E94290A8C2F0E94690DDB
:1017500067C0D23F21F128F4D03F41F0D13FC1F022
:1017600043C0D33F19F1D43F79F03EC0112341F07B
:10177000053008F051C08C2F8F710E948E0D4CC027
:10178000063008F049C0F7CF8091340282FF18C0BC
:10179000112339F08C2F8F710E94480D3DC0112309
:1017A000C9F38C2F8F710E94690D36C0112329F067
:1017B0008C2F8F710E94330D2FC00E942E0D2CC0D4
:1017C000112349F0CF718C2F0E94480D63E08C2FBC
:1017D0000E94651221C081E00E9480120230E0F078
:1017E00082E00E94801218C0112331F0002391F290
:1017F0008D2F0E94160910C0002399F2D93349F4A5
:101800001FEF27EE33E0115020403040E1F700C0D9
:1018100000008D2F0E94A30988EF8C0D843020F4E6
:101820000E9450240E948408DD20C9F00E94D31138
:1018300080FD15C0F70112820E94CD110E94480D53
:10184000C7010E94500C0E94CD11DF91CF911F91D2
:101850000F91FF90EF90DF90CF900C94690DDF9186
:10186000CF911F910F91FF90EF90DF90CF9008954F
:101870000F931F93CF93DF93EC01688179818A8165
:101880000E94890E8C010E94E50D0E94D60CB801C1
:10189000CE010E94300ADF91CF911F910F910895E0
:1018A000CF93DF93EC01988189812B813C81232B9D
:1018B00031F08F3F31F481E09F3F19F403C081E0A4
:1018C00001C080E080FD1DC0CE010E94EA078111A9
:1018D00010C00E94D7118823A1F08A81882389F043
:1018E0008091340282FD0DC082E0DF91CF910C9493
:1018F0008012CE010E94380CCE01DF91CF910C9462
:10190000CB07DF91CF9108950E94FE110C94201215
:1019100080910201909103010E94AB250C94840CEC
:101920000E94EE110C94880C92959F70963079F07D
:1019300010F4925001C09A50923068F4803F69F0E0
:1019400018F4883E40F409C0843F29F406C0883E5C
:1019500020F0813F11F080E0089581E00895FC01BE
:10196000808191810E947E0E0E94940C0895CF93F5
:10197000DF9300D000D01F92CDB7DEB70F900F904D
:101980000F900F900F90DF91CF910895CF93DF9339
:1019900000D000D000D0CDB7DEB726960FB6F894B1
:1019A000DEBF0FBECDBFDF91CF910895089508959A
:1019B0000C94D70C0C94D80C0E94DA0C609367013D
:1019C000709368018093690190936A010C94840C70
:1019D0000C94DC0C0F931F93009167011091680128
:1019E0002091690130916A01602B712B822B932B1E
:1019F0001F910F910C94DC0C0F931F9300916701C2
:101A0000109168012091690130916A01602371236E
:101A1000822393231F910F910C94DC0C0F931F933F
:101A200000916701109168012091690130916A016C
:101A300060277127822793271F910F910C94DC0C4C
:101A40000C94D70C0E94200D609363017093640185
:101A500080936501909366010C94840C60E070E0C3
:101A6000CB010C94220D0F931F9341E050E060E0F6
:101A700070E08A019B0104C0000F111F221F331F59
:101A80008A95D2F7C901B8011F910F910C94220DCC
:101A90000F931F9341E050E060E070E004C0440FFA
:101AA000551F661F771F8A95D2F780916301909129
:101AB0006401A0916501B09166018A019B01082B28
:101AC000192B2A2B3B2BC901B8011F910F910C94A4
:101AD000220D0F931F9341E050E060E070E004C0DE
:101AE000440F551F661F771F8A95D2F74095509572
:101AF000609570958091630190916401A09165015A
:101B0000B09166018A019B01082319232A233B23F4
:101B1000C901B8011F910F910C94220D0F931F93CF
:101B200041E050E060E070E004C0440F551F661FC4
:101B3000771F8A95D2F78091630190916401A091FB
:101B40006501B09166018A019B01082719272A27A0
:101B50003B27C901B8011F910F910C94220D0F93DF
:101B60001F930091630110916401209165013091F0
:101B70006601602B712B822B932B1F910F910C947C
:101B8000220D0F931F930091630110916401209126
:101B900065013091660160237123822393231F9195
:101BA0000F910C94220D0F931F93009163011091DC
:101BB00064012091650130916601602771278227B9
:101BC00093271F910F910C94220D0895262F890FB2
:101BD000982F9770A1E001C0AA0F9A95EAF7869511
:101BE0008695869590E065E070E00E94C52DFC0129
:101BF000E25AFE4F40E050E0622F70E090819B017E
:101C0000042E02C0369527950A94E2F7217021959B
:101C100029272A23292721934F5F5F4F45305105FC
:101C200069F70895890FA82FA770869586958695E0
:101C300090E065E070E00E94C52DBC0140E050E0FE
:101C400080E0FB01E40FF51FE25AFE4F208130E0F7
:101C50000A2E02C0369527950A94E2F721703327A1
:101C6000042E01C0220F0A94EAF7822B4F5F5F4FC8
:101C70004530510531F70895BF92CF92DF92EF9230
:101C8000FF920F931F93CF93DF938C01C09063015A
:101C9000D0906401E0906501F09066018091670149
:101CA00090916801A0916901B0916A01C82AD92A6E
:101CB000EA2AFB2ACFE1D0E0D701C6010C2E04C0EE
:101CC000B695A795979587950A94D2F780FD04C09D
:101CD000219790F7B12C07C0BC2EB8018C2F0E9421
:101CE00047150197A9F38B2DDF91CF911F910F918C
:101CF000FF90EF90DF90CF90BF900895CF93DF9348
:101D0000EC010E943C0EBE010E944715DF91CF916D
:101D100008951F93CF93DF93EB0190915D01992379
:101D200021F0CB010E947E0E13C0882349F0CB0125
:101D30000E943C0E182F682FCE010E94E60D04C0B1
:101D4000CB010E94120E182FBE01812F0E94471551
:101D5000DF91CF911F910895CF93DF93C0916B01D5
:101D600080916C01C817A1F0D0E0CE0166E070E070
:101D70000E94C52DFC01E359FE4F408151816281D3
:101D80007381848195810E94C60C2196C770E8CF2B
:101D9000DF91CF91089540919D0150919E016091F6
:101DA0009F017091A0018091A1019091A2010C94DA
:101DB000C60CFF920F931F93CF93DF938091A201E4
:101DC00082958F7009F062C080919F01882309F489
:101DD0005DC020916B01F0906C0110919D0100910C
:101DE0009E01A091A001B091A10181E01F3F09F0E7
:101DF00080E0C0910001D0910101482F2F1509F416
:101E000045C0109721F00F3F21F080E003C081E032
:101E100001C0842F30E080FD35C0C90166E070E06C
:101E20000E94C52DFC01E359FE4F818180132AC019
:101E30008081811327C08281811124C08381948194
:101E40008A1B9B0B8C179D07E8F48091A2018F7071
:101E500080618093A201C90166E070E00E94C52DF7
:101E6000FC01EE58FE4F90819F70906190838DE948
:101E700091E00E94500CDF91CF911F910F91FF9044
:101E80000C94AC0E2F5F3F4F2770B8CFDF91CF91EE
:101E90001F910F91FF9008959F92AF92BF92CF92A2
:101EA000DF92EF92FF920F931F93CF93DF93CDB703
:101EB000DEB761970FB6F894DEBF0FBECDBF8C01C1
:101EC00085E0F801DE011D9601900D928A95E1F7FB
:101ED000F801E28090919D0130919E016091A001F6
:101EE0007091A1016115710531F03F3F31F481E03E
:101EF0009F3F19F403C081E001C080E0F82FF1702A
:101F00009F2E80FD47C1F80140812181A380B480CC
:101F10008DE9C82E81E0D82EF0909F01F501E61BD7
:101F2000F70B6091000170910101FF2009F4DCC002
:101F30008091A201582F507FE617F70708F096C04E
:101F4000511155C0231313C0491311C0FE2CE110C9
:101F50000EC08F7080618093A2010E94CB0EC601DB
:101F60000E94500C8091A201F801858350C1AB28DA
:101F700031F02F3F31F481E04F3F19F403C081E08D
:101F800001C080E080FD03C081E08E2502C080E0BA
:101F900090E0F82FF170FF2E80FF1FC0E0916B01E1
:101FA00030916C01E31709F410C1F0E0CF0166E055
:101FB00070E00E94C52DDC01A359BE4F11968C9193
:101FC0001197281307C08C91481304C012968C9166
:101FD000E81203C03196E770E5CFFE2CEE2009F43D
:101FE00016C18091A20181608093A20154C0231385
:101FF00006C0491304C0E11002C0F80199C0C8012D
:102000000E94AF0C882361F1EE2051F12091A201D2
:10201000822F82958F7090E0029774F080919D01DD
:1020200090919E0198878F831986BB86AA862C87FC
:10203000CE0107960E94500C86E0F801ADE9B1E0B0
:1020400001900D928A95E1F70E94D90E0E94CB0E65
:102050000AC0231711F1C8010E94AF0C81112CC0D6
:10206000C8010E94500CFF24F394D1C05111F1CF4C
:102070007A2DB98AA88A522F6E2D89890E94B70CB1
:102080008DE991E00E94500C86E0F60111928A954C
:10209000E9F70E94CB0EF12CBAC04913DCCFE11056
:1020A000DACFF8018583C8010E94500C86E0F60162
:1020B00011928A95E9F7ABC0EE2091F22091A2012E
:1020C000822F82958F7090E002970CF4B5CF8091AB
:1020D0009D0190919E019A8389831B82BD82AC826F
:1020E0002E83CE010196A6CFE617F70708F044C06D
:1020F000FE2CEE2009F4B4CF231330C049132EC0B8
:102100002091A20120FD21C0822F82958F70482F3F
:1021100050E041155105C9F0F80125834F305105B4
:1021200041F08F5F982F9295907F822F8F70892B2F
:102130008583C8010E94500C86E0F801ADE9B1E04A
:1021400001900D928A95E1F73DC086E0F801ADE976
:10215000B1E001900D928A95E1F759C0C8010E9443
:10216000AF0C811169CF8091A20181608093A2019F
:10217000C8010E94500C4BC07A2DB98AA88A522FF0
:102180006E2D89890E94B70C86E0F60111928A951E
:10219000E9F718C0EE2009F463CFC8010E94AF0C24
:1021A000F82E882309F45CCF86E0F801ADE9B1E0B0
:1021B00001900D928A95E1F78DE991E00E94100956
:1021C0000E94D90E0E94CB0E22C04D872E878D858E
:1021D0009E850E947E0E292F22952F70223028F492
:1021E0009F7039F0811105C00BC0243028F49F7016
:1021F00049F4805E883020F0C8010E94500C9F2C6A
:10220000F92C05C0F8019581907F99F7F9CF8F2DB2
:1022100061960FB6F894DEBF0FBECDBFDF91CF91B0
:102220001F910F91FF90EF90DF90CF90BF90AF90F4
:102230009F900895CF93DF93CDB7DEB72C970FB65D
:10224000F894DEBF0FBECDBF4F83588769877A876A
:102250008B879C87CE0107960E944C0F8823D1F074
:102260009F8188852A853B85232B31F08F3F31F470
:1022700081E09F3F19F403C081E001C080E080FD50
:102280006FC04F81588569857A858B859C850E94B2
:10229000C60C66C086E0FE013796DE0111960190FD
:1022A0000D928A95E1F7FF81E8856A857B85611546
:1022B000710531F0EF3F31F481E0FF3F19F403C0C5
:1022C00081E001C080E080FD4BC080916C0190E016
:1022D0009C012F5F3F4F2770332740916B0150E0E7
:1022E0002417350709F443C0F983EA837D836C839F
:1022F00066E070E00E94C52DDC01A359BE4F96E058
:10230000FE01319601900D929A95E1F720936C01B0
:102310000E94AC0E25C090E066E070E00E94C52DE2
:1023200083599E4F0E944C0F882371F180916B015D
:1023300090E066E070E00E94C52DFC01E359FE4F7D
:102340004081518162817381848195810E94C60C94
:1023500080916B0190E001968770992780936B01C3
:1023600080916B0190916C018913D5CF0DC00E94B3
:10237000900C10926C0110926B01EDE9F1E086E097
:10238000DF011D928A95E9F72C960FB6F894DEBF0F
:102390000FBECDBFDF91CF9108958091C301859588
:1023A0008595859508958091C301877008959091D2
:1023B000C301977081E009F480E008958091E601FF
:1023C00008959091E601892B8093E6010895809508
:1023D0009091E60189238093E60108951092E60129
:1023E00008959091E501892B8093E50108958095EA
:1023F0009091E50189238093E50108951092E5010C
:1024000008958091C401089508950C9404120C94C9
:1024100005129091340292FD08C09091C401981762
:1024200021F08093C4010C94071208958091C40197
:10243000882329F01092C40180E00C9407120895BB
:10244000CF93DF93E0910201F09103018091E601C7
:102450008083E0910201F091030190818091E50178
:10246000892B80838091C401882381F0E09102014F
:10247000F09103019081892B8083809102019091DA
:1024800003010E94DD2481110E941612C0910201F5
:10249000D091030140E250E063EA71E0CE010E9476
:1024A000582E892B69F080E2FE01A3EAB1E0019089
:1024B0000D928A95E1F7CE01DF91CF910C945C24C7
:1024C000DF91CF9108950C9404129091340292FD03
:1024D00010C0982F990F990F990F692B6093C30122
:1024E0000E94480D8091C3018595859585950C9432
:1024F00063120C94480D1092C30180E00C94631297
:102500002091C301809582238093C301982F9770F7
:1025100099F430E0482F082E000C550B241735078E
:1025200059F09091340292FD07C085958595859567
:102530000E94690D0C947B120895CF939091340200
:1025400092FB222720F92817F9F0C82F892FC0FB0A
:1025500082F98093340280913302909134020E9478
:10256000F91282E00E9480128091F10180FF0CC07C
:102570001F92CF9387E591E09F938F930E947B07F3
:102580000F900F900F900F90CF910895809134028B
:1025900082FB882780F991E089270C949D1281E0C5
:1025A0000C949D1280E00C949D1280E090E00E94BB
:1025B000732E21E0893E9E4F09F020E0822F08957E
:1025C00082E090E00C94652E83E090E00C94652E00
:1025D000CF9384E090E00E94652EC82F82E290E0C5
:1025E0000E94652E2C2F30E0A901582BCA01CF91F3
:1025F0000895CF93C92F682F84E090E00E94792E30
:102600006C2F82E290E0CF910C94792EAB01BC014B
:102610008FE090E00C948B2EAB01BC0183E190E045
:102620000C948B2E60E070E0CB010C940C1360E0F6
:1026300070E0CB010E9406130C94121369EE7EEF3A
:1026400080E090E00E94972E60E082E090E00E949F
:10265000792E60E083E090E00E94792E109267016D
:10266000109268011092690110926A0160E084E0A2
:1026700090E00E94792E60E082E290E00E94792E44
:1026800060E085E090E00E94792E60E086E090E0D6
:102690000E94792E6FEF87E090E00E94792E40E053
:1026A00050E0BA0188E090E00E948B2E60E08DE05F
:1026B00090E00E94792E40E050E0BA0188E190E07D
:1026C0000E948B2E60E087E190E00E94792E40E02E
:1026D00050E0BA018CE190E00E948B2E60E070E047
:1026E00080E290E00E94972E40E050E0BA0188E13D
:1026F00090E00E948B2E0C9417130C941E13682FDD
:102700008EE090E00C94792E0E9466266093ED0195
:102710007093EE018093EF019093F0016093E901D3
:102720007093EA018093EB019093EC01089581E0AE
:1027300008950C94971308950C949B130C949B1379
:102740000C949E130C949B130C94A2130C949B1347
:1027500087E498E20E9446240E94A6130C94A413D6
:102760000E949C130C949B130E9424160C948308C3
:102770000E9451260E9407170E94B4130E94E81D70
:10278000E3E3F2E08081806880838091330290915E
:1027900034020E94F9120C94A013AF92BF92CF9210
:1027A000DF92EF92FF920F931F93CF93DF93CDB7FA
:1027B000DEB72A970FB6F894DEBF0FBECDBF0E94DA
:1027C0001617D82E81110E94841387EEA82E81E05F
:1027D000B82E00E010E0C02E802F0E944816F82E80
:1027E000F501E1905F01E82621F18091F10181FD81
:1027F0000E944E16E0FE1DC00E949913882389F0A6
:102800001E82CF828F2D817088870E945A26816018
:10281000782F9A8789874E815F8168858A850E9493
:10282000C608F801E951FE4F908181E08927808335
:1028300015C00F5F1F4F0230110569F68FEF8983B6
:102840008A831B820E945A268160782F9D838C8305
:1028500049815A816B818D810E94C60881E0D11027
:1028600001C080E02A960FB6F894DEBF0FBECDBF40
:10287000DF91CF911F910F91FF90EF90DF90CF905C
:10288000BF90AF9008950E94CD130E94971E0C94A4
:102890009408CF93DF930E944C15EC01811523E53A
:1028A0009207A0F5811532E5930708F0A2C08115C3
:1028B00040E29407C0F4811551E0950708F0D3C0B9
:1028C000853A910550F48430910508F0CCC0019709
:1028D00009F0C6C081E090E0C7C0805E910908970A
:1028E00008F4C1C0BDC0C11581E5D80708F07BC0A0
:1028F000C11520E5D20708F052C0C11530E4D30756
:1029000008F4AEC0DF70CE01906AAEC0811546E516
:10291000940708F5811555E5950708F087C0C1159E
:1029200084E5D80708F07CC09E012370332781E03E
:1029300090E002C0880F991F2A95E2F7C695C695C8
:10294000D0E065E0CC0FDD1F6A95E1F7C82BD92BED
:10295000CE019A6889C081152AE5920780F4811515
:1029600039E5930708F06BC0811548E5940708F432
:1029700077C0D82FCC27CE01806F906A75C0905653
:102980008115904208F06CC08D2F8F710E94E01568
:10299000DD27D0628F71AE01582BCA0165C0CE0110
:1029A000F4E096958795FA95E1F7282F23703C2F50
:1029B000337081E090E002C0880F991F3A95E2F7EA
:1029C0009C68AC01522B9C2F9F7096959695892FF1
:1029D00090E0EC01A5E0CC0FDD1FAA95E1F7CA015C
:1029E0008C2B9D2B41C0DC2FCC27CE01816F906AB0
:1029F0003BC09C012370332781E090E002C0880F28
:102A0000991F2A95E2F7C695C695D0E075E0CC0FE0
:102A1000DD1F7A95E1F7C82BD92BCE019C6824C025
:102A2000DC2FCC27CE01846F906A1EC00E94E01577
:102A30008F7190E0D82FCC27CE01906215C08F7097
:102A40000E94E01594E0D695C7959A95E1F7CF706E
:102A5000D0E0DC2FCC27D0699E01282BC90104C00F
:102A600080E090E001C0CE01DF91CF910895E62F84
:102A7000F0E0E70FF11D90E0880F991FE80FF91FB4
:102A8000EE0FFF1FE25EFE4F8591949108950E9424
:102A900037150E94491408958238910569F1B0F400
:102AA0008133910509F46DC048F48932910509F428
:102AB00063C08A32910509F469C008958533910590
:102AC00009F455C089339105B9F00895833E910505
:102AD00069F138F4803E9105B1F0823E910509F12B
:102AE0000895863E9105A9F1873E9105B9F1843E8E
:102AF000910509F064C023C02091330220FD4FC02E
:102B000021FD4DC008958091330280FD44C0809125
:102B1000340280FF44C08091330284FD42C083EEC2
:102B20004DC08091330282FF38C0F5CF80913302CF
:102B300082FD33C08091340280FD31C0ECCF8091A2
:102B4000340281FF32C08091330284FD2AC087EEB7
:102B500035C08091330283FF26C0F5CF80913302C8
:102B600083FD21C08091340281FD1FC0ECCF809194
:102B7000330285FD1CC01DC08091330285FD19C044
:102B800016C08091330286FD16C017C080913302B3
:102B900086FD13C010C089E311C082EE0FC080EE25
:102BA0000DC080E00BC086EE09C084EE07C089E24C
:102BB00005C085E303C08AE201C081E390E0089587
:102BC0009091330292FF0DC0282F2871283019F4FC
:102BD000877F846006C0282F2471243011F48B7FF6
:102BE000886093FF0DC0282F2871283119F4877E43
:102BF000846106C0282F2471243111F48B7E8861F2
:102C00002091340220FF0DC0382F3871383019F46C
:102C1000877F816006C0382F3171313011F48E7F8B
:102C2000886021FF0DC0282F2871283119F4877E74
:102C3000816106C0282F2171213111F48E7E8861B7
:102C400094FD877E089508950E94D512811102C0D7
:102C50000E947D130E94E0128093F1010E94E8120D
:102C600090933402809333020E9423160E94E41250
:102C7000682F70E080E090E00E94E80C60916301B2
:102C80007091640180916501909166010C94200D12
:102C9000E82FF0E0E95CFD4F80810895CF92DF924C
:102CA000EF92FF920F931F93CF93DF938BE791E007
:102CB0000E94E20687E3E82E82E0F82EC0E0D0E032
:102CC00096E7C92E91E0D92E0EE611E0DF93CF935F
:102CD000DF92CF920E947B0783E791E00E94E20699
:102CE000F70181917F010E946A081F928F931F93C1
:102CF0000F930E947B078CE691E00E94E2062196EA
:102D00008DB79EB708960FB6F8949EBF0FBE8DBFC5
:102D1000C230D105D9F6DF91CF911F910F91FF906D
:102D2000EF90DF90CF90089580EA8A95F1F70895AB
:102D300000C008950C94941608950C949C160C945D
:102D40009D160C949C160C94A116F894E82FE2950D
:102D5000EF70F0E031A1282F2F7081E090E001C0EA
:102D6000880F2A95EAF7982F9095932391A392A123
:102D7000892B82A37894089583E90E94A51685E69D
:102D80000E94A51682E90C94A5160F931F93CF936A
:102D9000DF938C01D62FC42FF894539A5B987894C4
:102DA0000E94981664E271E0F801A8014E5F5F4F3F
:102DB00010E03C2F3095DB012D91BD012F3FA9F094
:102DC000822F82958F7090E0DC0190968C9190E03C
:102DD0002F7002C0959587952A95E2F780FD05C072
:102DE00080818C2B808311E003C0808183238083CA
:102DF0003196E417F507F9F683E90E94A516612FCD
:102E00008D2FDF91CF911F910F910C949A160E94F4
:102E1000BC161092380210923702109236021092AD
:102E2000350282E00E944A170C94D6071F93CF9375
:102E3000DF9300D0CDB7DEB71A82198241E060E09F
:102E4000CE0101960E94C51642E050E0BE016F5FC0
:102E50007F4F85E392E00E94582E11E0009709F41D
:102E600010E0892B31F089819A819093360280930A
:102E70003502212F42E067E372E085E392E00E9491
:102E80004B170E94D807812F0F900F90DF91CF91A1
:102E90001F9108950895FF920F931F93CF93DF938F
:102EA0008C01F62ED72FC42F222349F081E0809386
:102EB000F4010E945A269093F3018093F2018091CD
:102EC000F4018823C1F08091F2019091F3010E94F6
:102ED0007226059780F0EF2DFD2FD8014C2F50E082
:102EE000CD01801B910B841795071CF48D91819364
:102EF000F7CF1092F401DF91CF911F910F91FF90C6
:102F000008950E94C3280E94B8130C94CF280E94F1
:102F1000D3280E9443140C94F1280E94F8250E94A3
:102F2000AA280E94A8130E9481170E9487170E9456
:102F3000B013FBCFEF92FF920F931F93CF93DF93CA
:102F4000E82F71110AC0442321F0F0E0E158FA4F54
:102F5000E4916E2F7E2F8E2F6CC0C62FD0E0072FEE
:102F600010E0282F30E0442329F0F901E158FA4F0E
:102F7000249130E0CE0166E070E00E94C52DEE2481
:102F8000EA94F12CB7010E94FB2DDB01CC0FDD1F71
:102F9000CB016BEA7FEF0E94C52D8C0F9D1FC82FC0
:102FA000CC0FC80FC701801B910BB9010E94C52D22
:102FB000E92F492FD0E0CE01B8010E94C52D692F1D
:102FC00070E0C701861B970BB9010E94C52DF92F30
:102FD000C7018C1B9D0BB8010E94C52D692F70E0A5
:102FE000C701861B970BB9010E94C52DA230B10500
:102FF00091F038F4109759F01197C1F48E2F7F2F6C
:103000000CC0A430B10579F050F0169779F4722F06
:10301000842FE92F0DC0892F7E2FE22F09C0822F28
:103020007E2FEF2F05C0822F792F02C0722F8F2F96
:103030006E2FDF91CF911F910F91FF90EF90089528
:1030400041E00E949A17089508950E94201808955B
:10305000CF93DF93762FE901682F842F0E942518E4
:10306000798368838A83DF91CF91089580913902B3
:10307000282F269530E02115310519F481708260E2
:1030800005C02532310524F08170886480933902AF
:10309000089588E090E00C946D2ECF92DF92EF922D
:1030A000FF926B017C010E943618B701A60188E0EF
:1030B00090E0FF90EF90DF90CF900C948B2EE9E39F
:1030C000F2E083E0808311828FEF82838383148216
:1030D00060817181828193810C944D188091F101FE
:1030E00080FF08C08FE494E09F938F930E947B073A
:1030F0000F900F908091F10180FF0FC080913902F5
:1031000081701F928F9382E394E09F938F930E942C
:103110007B070F900F900F900F908091F10180FF2F
:103120000FC08091390286951F928F9387E194E0BA
:103130009F938F930E947B070F900F900F900F909B
:103140008091F10180FF0EC080913A021F928F930F
:103150008DEF93E09F938F930E947B070F900F90CA
:103160000F900F908091F10180FF0EC080913B0283
:103170001F928F9383EE93E09F938F930E947B0720
:103180000F900F900F900F908091F10180FF0EC073
:1031900080913C021F928F9389EC93E09F938F93D1
:1031A0000E947B070F900F900F900F908091F1017C
:1031B00080FF0EC080913D021F928F938DEA93E0B5
:1031C0009F938F930E947B070F900F900F900F900B
:1031D00008958091390280FF02C08695089580E0AD
:1031E000089590913D02933018F49F5F90933D02B3
:1031F000882351F06091390270913A0280913B022C
:1032000090913C020C944D18089581E00C94F118B3
:1032100090913D02992319F0915090933D0288239B
:1032200051F06091390270913A0280913B02909185
:103230003C020C944D18089581E00C94081970E03C
:103240000C941420309108018091390280FF0CC049
:103250008091070190E063E070E00E94C52D632F2C
:10326000825C9D4F0C941F192091090140910A0125
:10327000241770F7822F90E063E070E00E94C52D64
:10328000FC01E25CFD4F1182108212822F5FF0CFB1
:10329000A82FB62F8091390280FF16C02091090116
:1032A00030910A01231770F4822F90E063E070E000
:1032B0000E94C52DFC01E25CFD4FA183B0834283D7
:1032C0002F5FF0CF0C9422190895CF93DF9300D095
:1032D0001F92CDB7DEB79091390290FF0AC09E01D0
:1032E0002F5F3F4F0E9428184B8169818A810E947D
:1032F00048190F900F900F90DF91CF910895CF93C1
:10330000DF93EC01EC81F0E0E658FB4F4491E9E3F8
:10331000F2E0628181810E9465198C818F5F8C83CC
:10332000DF91CF910895CF93DF93EC01E9E3F2E0D1
:10333000438162818C810E9465198C818F5F8C83AF
:10334000DF91CF9108950F931F93CF93DF9300D018
:103350001F92CDB7DEB78C018091F50181110AC0B3
:103360009E012F5F3F4F4FEF6FEF0E9428188A8119
:103370008093F501F8018481813051F028F082308A
:1033800061F44091F5010AC08091F50140E007C069
:103390006091F50140E080E003C040E080E060E043
:1033A0000E944819F801848190E0019663E070E082
:1033B0000E940F2E84830F900F900F90DF91CF917A
:1033C0001F910F9108954F925F926F927F928F920B
:1033D0009F92AF92BF92CF92DF92EF92FF920F93A4
:1033E0001F93CF93DF9300D01F92CDB7DEB7182F76
:1033F000D62E042F622E9091390290FFB3C0E92F90
:10340000E695AE2FB0E0AA5DBE4F8C918093FF0190
:103410009E7F923061F49E012F5F3F4F812F0E946B
:1034200028184B8169818A810E94481961C08230C5
:1034300019F400913C025CC0863019F410913A02F4
:1034400057C08930D9F3893109F052C0E9512E2F84
:103450002170722E81E0C22EC826E695F0E0E65873
:10346000FA4FE590F490412CFF2488E0A82E82E0EA
:10347000B82E20910B014216C8F5842C912CC40162
:10348000B7010E94C52D622F70E00E94FB2D512EC6
:10349000711002C0560E01C0561A8091F10180FFD2
:1034A00011C0FF92EF921F92CF921F925F921F92D4
:1034B0004F92BF92AF920E947B070FB6F894DEBF87
:1034C0000FBECDBF809109019401280F311DC901A4
:1034D00063E070E00E94C52D9C01225C3D4F402FAF
:1034E0006D2D852D0E9428184394C3CF0E94221968
:1034F00010933A02D0923B0200933C026620E9F01E
:103500006091390270913A0280913B0290913C02A5
:103510000E944D188091F10180FF24C080913C02EF
:103520001F928F9380913B021F928F9380913A025A
:103530001F928F9383EE91E00CC08091F10180FF88
:1035400011C01F920F931F92DF921F921F938CEB5B
:1035500091E09F938F930E947B070FB6F894DEBF94
:103560000FBECDBF0F900F900F90DF91CF911F91A5
:103570000F91FF90EF90DF90CF90BF90AF909F9012
:103580008F907F906F905F904F900895E9E3F2E005
:103590009181282F4381628186E0890F0C94E31981
:1035A00081E00C94C61AE9E3F2E09181282F43816F
:1035B00062818AEF890F0C94E31981E00C94D31A8D
:1035C000E9E3F2E0628124E0620F08F46FEF282F54
:1035D000438181810C94E31981E00C94E01AE9E3C2
:1035E000F2E0628124E0621B08F460E0282F43814E
:1035F00081810C94E31981E00C94EF1AE9E3F2E085
:1036000043812AE0420F08F44FEF282F6281818125
:103610000C94E31981E00C94FE1AE9E3F2E0438193
:103620002AE0421B08F440E0282F628181810C943B
:10363000E31981E00C940D1B20E00C94E319EF9248
:10364000FF921F93CF93DF93EC0110E0EE24EA94F6
:10365000F12C30910B01131700F520910901812FF6
:1036600090E0820F911D63E070E00E94C52DFC0187
:10367000E25CFD4F632F70E0C7010E940F2E812F87
:103680000E94BC2D9C819F0140913C0260913B02B5
:10369000890F0E9428181F5FDCCF0E9422199A818F
:1036A0008C8190FF02C08F5F01C081508C83DF91BD
:1036B000CF911F91FF90EF900895BF92CF92DF922C
:1036C000EF92FF920F931F93CF93DF93FC018281C0
:1036D00080FF02C0DFEF01C0D1E0C0E080910B01AC
:1036E000C81708F040C080910901CC2ED12C96015A
:1036F000280F311DC90163E070E00E94C52D825C76
:103700009D4F7C01FC0111821082128204E010E0C6
:10371000B12C8091F7018B0D853014F0837005C0BA
:1037200087FF03C090910B01890F082E000C990BA5
:10373000C816D90691F480913C0290E0B8010E942D
:10374000C52D95958795959587959701482F6091FB
:103750003B0280913A020E942818BD0E01501109C7
:10376000C1F6CF5FBBCF0E9422198091F701D13003
:1037700031F4811102C080910B01815007C090E0AB
:10378000019660910B0170E00E940F2E8093F7016B
:10379000DF91CF911F910F91FF90EF90DF90CF902D
:1037A000BF900895CF932091090130910A0123170A
:1037B00070F4822F90E063E070E00E94C52DFC0160
:1037C000E25CFD4F1182108212822F5FF0CFC0E0C9
:1037D00060910B01C61790F5EC2FF0E070E0CF017F
:1037E0000E940F2E90910901890F2091F601022E5F
:1037F000000C330B90E063E070E00E94C52DE217EF
:10380000F307A4F020910601022E000C330B2E17B3
:103810003F0764F09C01225C3D4F40913C02609167
:103820003B0280913A020E94281806C0FC01E25C2B
:10383000FD4F118210821282CF5FCACF0E942219DF
:10384000209105018091F601820F8093F6019091FD
:103850000601920F9093060119165CF4082E000CD5
:10386000990B40910B0150E0415051098417950785
:103870001CF0219520930501CF9108954F925F92FE
:103880006F927F928F929F92AF92BF92CF92DF9270
:10389000EF92FF920F931F93CF93DF938C01FC0164
:1038A000C481CC2ED12CE12CF12CA7019601C701AB
:1038B000B6010E94D62DA70196010E94D62D4B017C
:1038C0005C0180E290E06C01CC1AD1080D2C000C58
:1038D000EE08FF0825E530E040E050E0C501B40106
:1038E0000E94D62D2B013C01A7019601C701B6010C
:1038F0000E94D62DA70196010E94D62D9B01AC01F6
:10390000280D391D4A1D5B1DC301B2010E94232EE3
:10391000D22F822F90E02A3230F025E530E0A90145
:10392000481B590BCA0163E070E00E94C52D97FD4A
:10393000019695958795C82FC095F12C85E5E82EC1
:10394000ED1A80910B01F816D0F4F1FC02C0EE2DB7
:1039500001C0ED2F209109018F2D90E0820F911D64
:1039600063E070E00E94C52D9C01225C3D4F4C2F0E
:1039700060913B028E2F0E942818F394E2CF0E94A0
:103980002219F8018481811102C091E003C08032C4
:1039900019F49FEF9093040190910401890FF801AD
:1039A0008483DF91CF911F910F91FF90EF90DF9073
:1039B000CF90BF90AF909F908F907F906F905F90CF
:1039C0004F9008950F931F93CF93DF93EC0100E086
:1039D00010E040910B01842F90E0081719072CF597
:1039E000809109019801280F311DC90163E070E041
:1039F0000E94C52D9C01225C3D4F469550E08C8174
:103A0000041715071CF4882331F002C0811103C08C
:103A100040913C0201C040E060913B0280913A023B
:103A20000E9428180F5F1F4FD4CF0E9422198C814B
:103A300090E00196817099278C83DF91CF911F913F
:103A40000F91089560913902669570E04BE050E067
:103A50008CE091E00E944B2E892B19F481E0809339
:103A600000020E945A269093F9018093F8018091F8
:103A7000F10180FF08C083EA91E09F938F930E9439
:103A80007B070F900F900895109200028091F10132
:103A900080FF08C08AE891E09F938F930E947B0784
:103AA0000F900F9008959091390290FF54C091703B
:103AB000811102C0926006C0853210F0986402C085
:103AC000880F982B909339026623B1F060913902E8
:103AD00070913A0280913B0290913C020E944D18F5
:103AE0008091F10180FF1BC08091390286951F9261
:103AF0008F9383EF92E00BC08091F10180FF0FC0A4
:103B00008091390286951F928F9385ED92E09F9365
:103B10008F930E947B070F900F900F900F906091F2
:103B20003902669570E04BE050E08CE091E00E9435
:103B30004B2E892B19F00E94441D02C00E94221DA9
:103B400081E08093FB0140913C0260913B028091B7
:103B50003A020C941C1B0895682F90913902969597
:103B600081E0890F853208F081E00C94531D81E0DB
:103B70000C94AC1D682F9091390296958FEF890FA8
:103B800009F484E20C94531D81E00C94BA1D61E0A9
:103B90000C94531D80913902816080933902809189
:103BA000F10180FF0DC01F9281E08F9387E692E0C4
:103BB0009F938F930E947B070F900F900F900F9011
:103BC0008091390286950C94C71D60E00C94531DBA
:103BD0008091FE01811160C08091F10180FF08C0D9
:103BE00086E993E09F938F930E947B070F900F903D
:103BF0008091F10180FF08C080E893E09F938F934C
:103C00000E947B070F900F900E94D512811110C067
:103C10008091F10180FF08C088E593E09F938F9326
:103C20000E947B070F900F900E947D130E945F18E7
:103C30000E9449186093390270933A0280933B02C4
:103C400090933C026E7FC1F48091F10180FF08C027
:103C50008FE093E09F938F930E947B070F900F90CC
:103C60000E945F180E9449186093390270933A02CB
:103C700080933B0290933C020E9436180E946E187B
:103C8000109200028091390280FF03C086950E9445
:103C9000E51D81E08093FE010895809139028E7FB9
:103CA000809339026091390270913A0280913B020F
:103CB00090913C020E944D188091F10180FF0FC04D
:103CC0008091390281701F928F938FE292E09F93CF
:103CD0008F930E947B070F900F900F900F900E9480
:103CE000441D2FEF80E792E0215080409040E1F7A3
:103CF00000C000000C9422198091F10180FF10C0D7
:103D000080913902809581701F928F938EE992E0A5
:103D10009F938F930E947B070F900F900F900F90AF
:103D20008091390280FD0C944D1E0C94CA1D0F9396
:103D30001F93CF93DF9380910002882309F485C0FD
:103D40008091FF01E0913902E695E81BE093FA01CA
:103D5000823049F4F0E0EA58FB4FE491CE2FD0E0F6
:103D60000FE719E149C0863049F4F0E0ED58FB4F08
:103D7000E491CE2FD0E003E919E13EC0893051F43F
:103D8000E695F0E0E059FB4FE491CE2FD0E00FE153
:103D90001BE132C08F3051F4E695F0E0E359FB4F60
:103DA000E491CE2FD0E00DE51BE126C0853149F42A
:103DB000F0E0E659FB4FE491CE2FD0E002ED1BE19D
:103DC0001BC0883181F0833239F4E8E6F4E0C59114
:103DD000D49103EA19E110C0843251F4C4EFD1E068
:103DE00002EE1CE109C0C8E2D0E00EE31CE104C011
:103DF000C0EDD7E004E218E18091FB01882361F077
:103E00001092FB010E945A269093F9018093F801C9
:103E10001092FD011092FC010E945A26E091F801D7
:103E2000F091F9018E1B9F0B8F3F9F4770F4EC0FB1
:103E3000FD1FF093F901E093F80188EF91E0F8019C
:103E4000DF91CF911F910F910994DF91CF911F9135
:103E50000F910895882311F0FA0101C0FB01099424
:103E6000CF93DF93C82FD62F0E94E9188C1740F00C
:103E70000E94E9188D1720F4DF91CF910C94B71DA3
:103E80008C2FDF91CF910C94C71D1F93CF93DF939D
:103E9000FB0112811111C3C0EC010E94DE1182727C
:103EA000CD3CFCE5DF0709F49AC0A8F5C73CECE57A
:103EB000DE0709F476C0A8F4C43C9CE5D90709F4F0
:103EC0005FC028F4C33CDC4509F457C054C0C53C6E
:103ED0009CE5D90709F459C0C63CDC4509F45CC02F
:103EE0004AC0CA3CFCE5DF0709F46AC050F4C83C8C
:103EF000ECE5DE0709F45AC0C93CDC4509F45BC0B7
:103F00003AC0CB3C9CE5D90709F45FC0CC3CDC450A
:103F100009F460C030C0C23DFCE5DF0709F46FC0A2
:103F200088F4CF3C9CE5D90709F460C008F45CC074
:103F3000C03DFCE5DF0709F45CC0C13DDC4509F488
:103F40005BC019C0C53D9CE5D90709F460C050F4B9
:103F5000C33DFCE5DF0709F455C0C43DDC4509F469
:103F600054C009C0C63D9CE5D90709F455C0CE35FB
:103F7000DD4509F454C011E052C00E947C1E4FC0C0
:103F800044EC5DE167EB7DE104C047EB5DE164EC8F
:103F90007DE10E942A1F43C04DED5AE160ED7AE1B8
:103FA000F8CF40ED5AE16DED7AE1F3CF4BEF5AE1F6
:103FB0006CEE7AE1EECF4CEE5AE16BEF7AE1E9CFAD
:103FC00049E15BE16AE07BE1E4CF4AE05BE169E182
:103FD0007BE1DFCF4CE159E165E079E1DACF45E003
:103FE00059E16CE179E1D5CF81E017C065E082E06D
:103FF00010C068E086E00DC06EE089E00AC064E1B0
:104000008FE007C067E185E104C088E106C062E295
:1040100089E10E94301F03C083E20E94C71D812FE7
:10402000DF91CF911F910895239A25B1277F35B154
:1040300038604FB7F894FC01CB0163E070E00E9458
:10404000C52D8E0F9F1FE817F90789F0519168E081
:1040500035B9000000C057FF25B9550F000000C05A
:1040600000C000C025B900C06A9591F7ECCF4FBFE2
:104070008FE594E00197F1F700C000000895CF9319
:10408000DF93EC01FB018281882309F43CC1C43039
:10409000FDE5DF0760F4CB3F9CE5D90788F49E017E
:1040A00022503C452431310508F02EC109C0C236EA
:1040B000EDE5DE0729F0C63AFDE5DF0709F024C18A
:1040C0000E94E8129093340280933302C1318CE550
:1040D000D80709F4C6C008F042C0C930ECE5DE07D5
:1040E00009F49BC000F5C5308CE5D80709F485C0FC
:1040F00078F4C330ECE5DE0709F478C008F07AC044
:10410000C230DC4509F0F5C0809133028160EFC018
:10411000C7309CE5D90709F478C008F07AC08091CF
:1041200033028061E4C0CD30FCE5DF0709F487C0CD
:1041300058F4CB309CE5D90709F479C008F07BC06E
:104140008091330288606FC0CF30FCE5DF0709F44F
:1041500080C008F082C080913302877FC8C0CE3F04
:104160009CE5D90709F471C000F5C531FCE5DF070E
:1041700009F485C068F4C3319CE5D90709F475C01A
:1041800008F095C00E94900C809133028F77AFC0E9
:10419000CC3FFCE5DF07A9F108F054C0CB3FDC457C
:1041A00009F0A7C08091340240C0C230EDE5DE07BF
:1041B00009F489C058F4C1158DE5D80709F45AC02F
:1041C00008F069C08091340282602FC0C236EDE5EC
:1041D000DE0709F47CC0C63AFDE5DF0709F481C0BB
:1041E000C330DD4509F085C080E06EC080913302A8
:1041F00082607DC08091330216C080913302886056
:1042000076C08091340282604FC080913302806218
:104210006EC08091330280646AC00E94900C8091CD
:104220003302806864C0846062C081603DC0809158
:1042300033028E7F5CC0809133028D7F58C08091A5
:10424000330216C08091340218C0809134028D7FF1
:104250002BC0809133028F7E4AC0809133028F7DC4
:1042600046C0809133028F7B42C080913302877FAA
:104270008B7F3DC0809134028D7F8E7F15C08091F1
:10428000330282FB222720F991E0922790FB82F9EA
:1042900090FB83F92CC080913402982F90959170F7
:1042A0008E7F892B90FB81F98093340222C00E947B
:1042B000900C8091330287FB222720F991E092270E
:1042C00090FB87F914C081E00E947F1312C0809197
:1042D000330284FB222720F991E0922790FB84F996
:1042E00006C080913302982F909590FB80F98093BF
:1042F000330280913302909134020E94F9120E949D
:10430000900C80E001C081E0DF91CF910895CF93C0
:10431000C82F1F928F9385E896E09F938F930E94FA
:104320007B0781E090E0A0E0B0E0BC01CD0104C0DB
:10433000660F771F881F991FCA95D2F70E94E80C55
:104340000F900F900F900F90CF910C94900CDF92E4
:10435000EF92FF920F931F93CF93DF93482F50E07C
:10436000FA013597EF33F10508F03FC1EA5BFF4FE3
:104370000C94452E0E94E4121F928F938FEB9AE0CB
:104380009F938F930E947B070E94E01283FB9927E3
:1043900090F91F929F9382FB992790F91F929F9308
:1043A00081FB992790F91F929F93982F91701F92EC
:1043B0009F931F928F9386E79AE09F938F930E941B
:1043C0007B070E94E81287FB222720F91F922F9378
:1043D00086FB222720F91F922F9385FB222720F9A5
:1043E0001F922F9384FB222720F91F922F9383FB88
:1043F000222720F91F922F9382FB222720F91F9258
:104400002F9391FB222720F91F922F93292F2170A0
:104410001F922F9381FB222720F91F922F93282F81
:1044200021701F922F939F938F9381E999E09F931F
:104430008F930E947B078DB79EB788960FB6F8942E
:104440009EBF0FBE8DBF06C08FE79BE00E94E206B5
:104450000E947D13C1E0CEC08FED97E074C08091C3
:10446000F101817F8E7F8093F10184EC97E00E94BF
:10447000E2068BE79BE00E94E20681E08093010266
:10448000E9CF8FE59BE00E94E2060E94DB07E2CFC6
:104490008091F101C82FC095C170C0FB80F9809355
:1044A000F101CC2319F083E59BE091C086E49BE009
:1044B0000E94E2068091F101897F877F8093F1015C
:1044C000C9CF9091F10191FBCC27C0F981E0C827B9
:1044D000892FC0FB81F98093F101CC2319F089E386
:1044E0009BE027C08BE29BE02EC09091F10192FBF4
:1044F000CC27C0F981E0C827892FC0FB82F98093BF
:10450000F101CC2319F08CE19BE013C08CE09BE01F
:104510001AC09091F10193FBCC27C0F981E0C82724
:10452000892FC0FB83F98093F101CC2351F080E007
:104530009BE00E94E2068091F10181608093F1018D
:1045400059C083EF9AE00E94E20684CF8EE097E0A4
:10455000FACF0E946626062FF72EE82ED92EC0919C
:104560003302C7FBCC27C0F910913202D09123014E
:104570000E945024DF92EF92FF920F931F92CF93ED
:104580001F921F931F92DF931F928F938AE896E0EA
:104590009F938F930E947B078DB79EB70E960FB6A1
:1045A000F8949EBF0FBE8DBF55CF0E94900C909186
:1045B000330297FBCC27C0F981E0C827892FC0FBC5
:1045C00087F980933302CC2329F089EE9AE00E9488
:1045D000E20610C08EED9AE0B6CF895303C08D512C
:1045E00001C080E00E94872135CF8CED9AE00E94C7
:1045F000E206C0E08C2FDF91CF911F910F91FF90C9
:10460000EF90DF90089580E008950C940323CF93FA
:10461000C82F80910102882319F0813031F038C011
:104620000E94DE118232B1F504C00E94DE11823296
:1046300061F48C2F0E940523811104C08C2F0E94ED
:10464000A72124C081E090E021C08C2F0E94032389
:1046500081111BC0C43189F018F4CB3029F010C08F
:10466000C93259F0C83361F484EC97E00E94E20645
:1046700081E896E00E94E20608C0109201020CC098
:104680008FE796E00E94E20607C081E0817006C0D5
:104690001092010280E002C080E0F8CFCF9108952F
:1046A000CF93DF9386319C4541F5EB010E94DE11EB
:1046B000982F8A812091020130910301882379F09B
:1046C0009A7A81E009F480E080930202911102C09D
:1046D00069E201C065E3C9010E9495250AC0809185
:1046E0000202811102C069E201C065E3C9010E94B2
:1046F000A0250E94201280E001C081E0DF91CF91CF
:1047000008950F931F93CF93DF93C42FD22FFC01F3
:1047100082818823C9F0409305020E945A26909313
:1047200004028093030280E28C0F883008F057C0A7
:10473000C77081E001C0880FCA95EAF7DF91CF9179
:104740001F910F910C94220A80910502481330C0EA
:1047500080910302909104020E947226883C910588
:1047600038F510E21D0FCD17B9F080E28C0F8830BC
:1047700040F4C77081E001C0880FCA95EAF70E9433
:10478000290A183028F581E09D2F977001C0880F05
:104790009A95EAF70E94220A802F0E94190A18307F
:1047A000F0F4D77081E001C0880FDA95EAF70AC00B
:1047B00080E28C0F883098F4C77081E001C0880FC8
:1047C000CA95EAF7DF91CF911F910F910C94290AB6
:1047D000802FDF91CF911F910F910C94190ADF91D7
:1047E000CF911F910F9108950F939C01CB01243F0E
:1047F0004CE5340731F188F4293DFCE53F07D9F059
:104800002A3D4CE5340779F1283D3C45A9F506E2FF
:1048100021EE41EE68ED7CE52BC0263FFCE53F072D
:10482000E1F0A8F0273F3C4539F507E225EE46EEDA
:1048300067EF7CE51DC007E225EE45EE69ED7CE5FE
:1048400017C006E221EE40EE64EF7CE511C007E2FE
:1048500025EE44EE65EF7CE50BC006E221EE42EE6C
:1048600066EF7CE505C008E221E045EE6AED7CE5F7
:104870000E94812380E008C0FC018281882319F016
:104880001092050201C081E00F91089590935B01A1
:1048900080935A01089590930B0280930A02089521
:1048A000E0910A02F0910B02309721F00190F08123
:1048B000E02D099480E00895EF92FF921F93CF932B
:1048C000DF93FC01A0910A02B0910B02109709F44A
:1048D00042C080912301882341F08091330287FFF9
:1048E00004C08081818386E08083EF011296ED9180
:1048F000FC911397CE0109958091F10182FF2BC0A5
:1049000080FF04C088E99BE00E94E20618E082E98B
:10491000E82E8BE0F82E8091F10180FF0BC088819A
:104920001F928F93FF92EF920E947B070F900F9040
:104930000F900F90115021961111EDCF8091F10140
:1049400080FF09C080E99BE0DF91CF911F91FF902C
:10495000EF900C94E206DF91CF911F91FF90EF90C2
:10496000089520910802309109022817390771F043
:104970009093090280930802E0910A02F0910B02E1
:10498000309721F00680F781E02D09940895209159
:104990000602309107022817390771F09093070239
:1049A00080930602E0910A02F0910B02309721F009
:1049B0000084F185E02D09940895FC0132968091E0
:1049C0002301882331F08091330287FF02C09EE1EA
:1049D00001C096E080E0915028F021912223D9F384
:1049E0008F5FF9CF0895662351F12091230122238F
:1049F000E9F02091330227FF19C0462F46954695CE
:104A000046954E31E0F4677021E030E002C0220F9D
:104A1000331F6A95E2F7FC01E40FF11D828190E0FB
:104A20002823392381E0232B69F409C0FC01329645
:104A300008962191621729F0E817F907D1F780E06D
:104A4000089581E008959C01FC0132969FEF80E07B
:104A50004191461789F09F3F19F4411101C0982FE9
:104A60008F5F8630A9F79F3F39F0F901E90FF11DFB
:104A700097FDFA956283089508959C012A5F3F4F40
:104A8000FC014281461301C01282019682179307EE
:104A9000B9F70895262F2695269526952E3170F480
:104AA000FC01E20FF11D677021E030E001C0220F30
:104AB0006A95EAF78281282B228308958091F1017B
:104AC00080FF0CC01F926F9388EC9BE09F938F93A5
:104AD0000E947B070F900F900F900F900895262F44
:104AE0002695269526952E3178F4FC01E20FF11DCE
:104AF000677021E030E001C0220F6A95EAF7209547
:104B000082812823228308958091F10180FF0CC0C7
:104B10001F926F938AEA9BE09F938F930E947B077B
:104B20000F900F900F900F90089520912301222352
:104B300029F02091330227FD0C944A250C9423255B
:104B400020912301222329F02091330227FD0C9488
:104B50006F250C943D2520912301FC0132962223E0
:104B600031F08091330287FF02C08EE101C086E000
:104B7000DF011D928A95E9F7089508950C94BD25EB
:104B800083E080930C020C94BE25811102C081E069
:104B900001C082E080930C020C94BE250C94C525C4
:104BA00081E080930C020C94BE250C94D0250895CE
:104BB0000C94D7250C94D8250C94D7250C94D72584
:104BC0000C94D7250E94DE250E9416170E94DC2532
:104BD00080E00E944816811108C081E00E944816BA
:104BE00091E0811103C090E001C091E0892F089508
:104BF00008951F920F920FB60F9211248F939F93D7
:104C0000AF93BF9380910D02811113C080914A022E
:104C100090914B02A0914C02B0914D024196A11D82
:104C2000B11D80934A0290934B02A0934C02B09323
:104C30004D02BF91AF919F918F910F900FBE0F903A
:104C40001F90189580915202843031F10E946208C1
:104C500010920D0220E488E190E00FB6F894A89538
:104C6000809360000FBE2093600083B7817F8460D3
:104C700083BF83B7816083BF7894889583B78E7F25
:104C800083BF0FB6F894A8958091600088618093E7
:104C90006000109260000FBE08950E94900C0C946A
:104CA000660882E084BD93E095BD9AEF97BD80933E
:104CB0006E0008952FB7F89480914A0290914B02AC
:104CC000A0914C02B0914D022FBF08952FB7F894D8
:104CD00060914A0270914B0280914C0290914D027A
:104CE0002FBF08959C014FB7F89480914A0290918C
:104CF0004B02A0914C02B0914D024FBF821B930B0F
:104D0000089578941F920F920FB60F9211248F93EB
:104D10009F93AF93BF9380914A0290914B02A091D1
:104D20004C02B0914D020196A11DB11D80934A0223
:104D300090934B02A0934C02B0934D02BF91AF9160
:104D40009F918F910F900FBE0F901F90189581E04B
:104D50008093E00080E28093D8001092C9008FE138
:104D60009EE40197F1F700C0000087E090EBDC01C2
:104D700080935B0290935C02A0935D02B0935E020D
:104D80009CE088E10FB6F894A895809360000FBE70
:104D900090936000FFCF80913102089508950895A7
:104DA000CF93DF9320912301222339F02091330206
:104DB00027FF03C060E222E002C068E021E0209308
:104DC000E9002FEF3091E800215035FD06C035EDA8
:104DD0003A95F1F700002111F5CF2091E80025FF69
:104DE0001DC0EC0180912301811105C040E050E01D
:104DF00068E070E003C070E040E050E0CE010E9447
:104E000060298091E8008E778093E80080E2FE01BF
:104E1000A1E1B2E001900D928A95E1F7DF91CF9187
:104E200008950895089582EF9BE00E94E2060C9495
:104E3000D5258EEE9BE00E94E20660914E0281E055
:104E4000611101C080E00C94C0258AEE9BE00E94B5
:104E5000E2069091520281E0943009F080E0609186
:104E60004E020C94C52520910F022F5F822F62E322
:104E70000E94EF2D992319F020930F0208951092AC
:104E80000F0280911002882371F1809152028430C8
:104E900041F58091E9008F702091EC00922F917084
:104EA00020FD90E8892B93E09093E9009091EB002E
:104EB00090FF14C09091EE0097FF10C09091E80011
:104EC00095FF03C01092F100F9CF9091E80090FF98
:104ED00005C09091E8009E779093E8008F708093D2
:104EE000E90010921002089542E061EC81E00E9416
:104EF000642A42E261EC82E00E94642A42E261ECB0
:104F000083E00E94642A9091520281E0943009F07B
:104F100080E060914E020C94CE2580915402833043
:104F200009F45DC030F4813071F0823009F496C02C
:104F300008958A3009F482C08B3009F468C0893042
:104F400009F0A4C020C080915302813A09F09EC0AC
:104F50008091E800877F8093E800809157029091CC
:104F60005802892B21F460E281E192E003C060E005
:104F700080E090E070E00E94AB298091E8008B77A0
:104F80008093E800089580915302813209F07EC039
:104F90008091570290915802029708F077C0809153
:104FA000E800877F8093E8008091E80082FD05C0DB
:104FB000809152028111F8CF69C08091F200823055
:104FC00031F48091F100813011F0863021F480912C
:104FD000F100809331028091E8008B7753C080917B
:104FE0005302813A09F052C08091570290915802C1
:104FF000892B09F04BC08091E800877F8093E800FF
:105000008091E80080FFFCCF8091230136C0809121
:1050100053028132D9F58091570290915802892B21
:10502000A9F58091E800877F8093E8000E94992A83
:1050300080915502809323010C94900C809153022F
:10504000813221F58091E800877F8093E8000E94FB
:10505000992A8091560280933202089580915302DA
:10506000813AA1F48091E800877F8093E8008091E5
:10507000E80080FFFCCF809132028093F1008091A4
:10508000E8008E778093E8000C94992A08959FB7E2
:10509000F894109210029FBF90915202943009F040
:1050A00057C09091E9009F703091EC00232F217040
:1050B00030FD20E8922B23E02093E9002091EB00C3
:1050C00020FF43C02091EE0027FF3FC020910E0239
:1050D000222321F02091E80025FF37C010920E0214
:1050E00026E03091E80035FD15C030915202343091
:1050F00061F53091EB0035FD28C0215021F481E0AD
:1051000080930E0222C0EFE9FFE03197F1F700C073
:105110000000E7CF8093F1008091E80085FD0AC090
:105120008091E80080FFFCCF8091E8008E7780932B
:10513000E80006C08FB7F89421E0209310028FBFDB
:105140009F709093E90080E008959F709093E9002C
:105150008FEF089584B7877F84BF0FB6F894A89522
:1051600080916000886180936000109260000FBEA3
:1051700090E080E80FB6F89480936100909361000E
:105180000FBE0C94D0250E94EB2A0E943E2BE2EE2B
:10519000F0E080818460808378940C94A12D87E175
:1051A00091E00C944B24809152028530C9F486EE34
:1051B0009BE00E94E20680915202853079F40E94C1
:1051C0002226809150028823B1F30E94E225882391
:1051D00091F30E944A290E94900CEDCF0C944D2629
:1051E000089508950C94F428292F3327233031058E
:1051F000C9F060F42130310581F02230310509F029
:1052000041C08BE590E02EE23CE040C02132310508
:10521000E1F02232310531F135C082E190E029E838
:105220003CE034C099278130910549F028F002977D
:1052300049F5E6EFFBE005C0EAE2FCE002C0E0E190
:10524000FCE0849190E09F0121C063307105D0F4AF
:10525000660F771FFB01EC5AFE4F2081318189E0F8
:1052600090E014C06330710568F4FB01EE0FFF1F7E
:10527000E25BFE4F20813181FB01E55BFE4F8081C7
:1052800090E004C080E090E020E030E0FA0131835B
:105290002083089584E089BD86E089BD09B400FEBD
:1052A000FDCF8091D8008F7D8093D8008091E00061
:1052B00082608093E0008091E00081FDFCCF089542
:1052C000CF92DF92EF92FF920F931F93CF93DF93D2
:1052D000EC018B017A010E94B82A811133C0E114DC
:1052E000F10439F0F70180819181081B190BC80F77
:1052F000D91FC12CD12C0115110519F18091E8009D
:1053000085FD16C08091E8008E778093E800E11457
:10531000F10449F0F70180819181C80ED91ED18234
:10532000C08285E00FC00E94B82A882321F30AC0FA
:1053300089918093F10001501109FFEFCF1ADF0A24
:10534000DACF80E0DF91CF911F910F91FF90EF9026
:10535000DF90CF9008952091590230915A0226177C
:10536000370748F06115710539F42091E8002E7770
:105370002093E80001C0B901FC0120E0611571052E
:1053800061F1809152028823D9F18530D9F1809161
:10539000E80083FD39C08091E80082FD2BC0809138
:1053A000E80080FFEBCF8091F20090E0611571057D
:1053B00051F08830910538F421912093F10061502B
:1053C00071090196F3CF21E0089709F020E0809160
:1053D000E8008E778093E800D1CF2111D2CF0AC0A8
:1053E00080915202882361F0853061F08091E8005D
:1053F00083FD0AC08091E80082FFF2CF80E008952B
:1054000082E0089583E0089581E008952091590293
:1054100030915A022617370748F06115710539F4A3
:105420002091E8002E772093E80001C0B901FC012B
:1054300020E06115710579F180915202882309F409
:105440003DC0853009F43CC08091E80083FD3AC03E
:105450008091E80082FD2CC08091E80080FFE9CFB8
:105460008091F20090E06115710559F08830910546
:1054700040F424912093F100319661507109019616
:10548000F2CF21E0089709F020E08091E8008E77C4
:105490008093E800CECF2111CFCF0AC08091520275
:1054A000882361F0853061F08091E80083FD0AC0B7
:1054B0008091E80082FFF2CF80E0089582E00895B5
:1054C00083E0089581E00895982F953068F59093D2
:1054D000E900981739F07091EC002091ED0050919F
:1054E000F00003C0242F762F50E021FD02C09F5F03
:1054F000ECCF3091EB003E7F3093EB003091ED002C
:105500003D7F3093ED003091EB0031603093EB0044
:105510007093EC002093ED005093F0002091EE008A
:1055200027FDE5CF80E008958F708093E90081E04A
:1055300008958091530287FF11C08091E80082FD99
:1055400005C0809152028111F8CF11C08091E8000E
:105550008B770BC080915202882349F08091E8003C
:1055600080FFF8CF8091E8008E778093E80008955F
:105570002091E4003091E50095E64091EC00842F05
:10558000817040FF23C08091E80080FD1DC08091A4
:105590005202882399F0853099F08091EB0085FDC7
:1055A00011C04091E4005091E5002417350729F31C
:1055B000915011F09A01E1CF84E0089582E00895BE
:1055C00083E0089581E0089580E008954091E80027
:1055D00042FFDDCF08950E94482B0E944B2BE0EE46
:1055E000F0E0808181608083E8EDF0E080818F775A
:1055F000808319BCE3E6F0E08081816080831092B3
:10560000510208950E94482B0E944B2B8091D80094
:105610008F778093D8008091D80080688093D800DD
:105620008091D8008F7D8093D80084E089BD86E08A
:1056300089BD09B400FEFDCF1092520210924E02B5
:105640001092500210924F0242E060E080E00E940F
:10565000642A8091E1008E7F8093E1008091E200D6
:1056600081608093E2008091E20088608093E20094
:105670008091E0008E7F8093E0000895E3E6F0E003
:1056800080818E7F808381E0809351020C94022B75
:105690001092E20008951092E10008951F920F9277
:1056A0000FB60F9211242F933F934F935F936F93F5
:1056B0007F938F939F93AF93BF93EF93FF938091CB
:1056C000E10082FF0BC08091E20082FF07C0809161
:1056D000E1008B7F8093E1000E9433278091E100FD
:1056E00080FF19C08091E20080FF15C08091E20028
:1056F0008E7F8093E2008091E20080618093E200DF
:105700008091D80080628093D80019BC85E0809396
:1057100052020E9419278091E10084FF30C08091DD
:10572000E20084FF2CC084E089BD86E089BD09B415
:1057300000FEFDCF8091D8008F7D8093D8008091AE
:10574000E1008F7E8093E1008091E2008F7E809364
:10575000E2008091E20081608093E20080914E023D
:10576000882311F084E007C08091E30087FD02C028
:1057700081E001C083E0809352020E94252780913E
:10578000E10083FF29C08091E20083FF25C0809162
:10579000E100877F8093E10082E0809352021092C3
:1057A0004E028091E1008E7F8093E1008091E200C3
:1057B0008E7F8093E2008091E20080618093E2001E
:1057C00042E060E080E00E94642A8091F0008860FE
:1057D0008093F0000E941327FF91EF91BF91AF914A
:1057E0009F918F917F916F915F914F913F912F91F9
:1057F0000F900FBE0F901F9018951F920F920FB62B
:105800000F9211242F933F934F935F936F937F9346
:105810008F939F93AF93BF93CF93DF93EF93FF93B8
:10582000C091E900CF708091EC00D82FD17080FD3D
:10583000D0E81092E9008091F000877F8093F0001B
:1058400078940E94412C1092E9008091F0008860C9
:105850008093F000CD2BCF70C093E900FF91EF91C2
:10586000DF91CF91BF91AF919F918F917F916F9178
:105870005F914F913F912F910F900FBE0F901F900E
:1058800018951F93CF93DF93CDB7DEB7AA970FB6C6
:10589000F894DEBF0FBECDBFE3E5F2E08091F100EA
:1058A000819322E0EB35F207C9F70E948D278091A2
:1058B000E80083FF2EC18091530290915402492F3A
:1058C00050E04A30510508F024C1FA01EB57FF4F70
:1058D0000C94452E803821F0823809F01AC108C096
:1058E00080914F0290915002992389F082600FC0FD
:1058F000809157028F70853008F00BC18093E900CA
:105900008091EB0085FB882780F91092E900909147
:10591000E800977F9093E8008093F1001092F100E7
:10592000D1C0282F2D7F09F0F4C0882319F08230D0
:1059300061F0EFC080915502813009F0EAC09330E8
:1059400009F080E0809350022EC0809155028111B1
:105950002AC0809157028F702FEF280F243008F053
:10596000D8C08093E9002091EB0020FF1CC0933049
:1059700021F48091EB00806214C09091EB00906163
:105980009093EB0021E030E0A90102C0440F551FC5
:105990008A95E2F74093EA001092EA008091EB00CA
:1059A00088608093EB001092E9008091E800877F87
:1059B0008093E8000E94992AACC08111AAC010917E
:1059C00055021F778091E3008078812B8093E3005C
:1059D0008091E800877F8093E8000E94992A809157
:1059E000E80080FFFCCF8091E30080688093E300B3
:1059F000111102C082E001C083E08093520289C08D
:105A00008058823008F085C08091550290915602EE
:105A10008C3D53E0950779F583E08A838AE2898398
:105A20004FB7F894DE01139620E03EE051E2E32FF9
:105A3000F0E050935700E49120FF03C0E295EF702F
:105A40003F5FEF708E2F90E0EA3010F0C79601C0F4
:105A5000C0968D939D932F5F243149F74FBF80915E
:105A6000E800877F8093E8006AE270E0CE0101964B
:105A70000E94AB2916C06091570270915802AE0186
:105A80004F5F5F4F0E94F228BC01892B09F441C08F
:105A90009091E800977F9093E80089819A810E9415
:105AA000062A8091E8008B778093E80032C0803826
:105AB00081F58091E800877F8093E80080914E0215
:105AC0008093F1008091E8008E7772CF811121C020
:105AD000809155029091560299270297D4F48091B3
:105AE000E800877F8093E8008091550280934E0202
:105AF0000E94992A80914E02811106C08091E30094
:105B000087FD02C081E001C084E0809352020E94C0
:105B100074278091E80083FF0AC08091E800877FA6
:105B20008093E8008091EB0080628093EB00AA965E
:105B30000FB6F894DEBF0FBECDBFDF91CF911F919E
:105B40000895CF93809152028823A1F0C091E9007B
:105B5000CF709091EC00892F817090FD80E8C82B68
:105B60001092E9008091E80083FD0E94412CCF70E3
:105B7000C093E900CF910895002480FD060E660FC2
:105B800011F08695D1F7802D08950024552704C083
:105B9000080E591F880F991F009729F07695679571
:105BA000B8F37105B9F7802D952F0895EE27FF27DB
:105BB000AA27BB2708C0A20FB31FE41FF51F220F9F
:105BC000331F441F551F969587957795679598F3D2
:105BD0007040A9F7009799F7BD01CF010895991B6F
:105BE00079E004C0991F961708F0961B881F7A95D4
:105BF000C9F780950895AA1BBB1B51E107C0AA1FD6
:105C0000BB1FA617B70710F0A61BB70B881F991F5D
:105C10005A95A9F780959095BC01CD01089597FB01
:105C2000072E16F4009407D077FD09D00E94FB2DB3
:105C300007FC05D03EF4909581959F4F089570958F
:105C400061957F4F0895A1E21A2EAA1BBB1BFD018F
:105C50000DC0AA1FBB1FEE1FFF1FA217B307E4074B
:105C6000F50720F0A21BB30BE40BF50B661F771FA3
:105C7000881F991F1A9469F7609570958095909583
:105C80009B01AC01BD01CF010895EE0FFF1F0590F0
:105C9000F491E02D0994FC014150504030F0019006
:105CA0000616D1F73197CF010895882799270895CF
:105CB000FB01DC0104C08D910190801921F4415059
:105CC0005040C8F7881B990B0895F999FECF92BDF3
:105CD00081BDF89A992780B50895A6E1B0E044E027
:105CE00050E00C949F2EA8E1B0E042E050E00C940C
:105CF0009F2E262FF999FECF92BD81BDF89A01976C
:105D000000B4021639F01FBA20BD0FB6F894FA9A03
:105D1000F99A0FBE08950396272F0E947A2E0E94AB
:105D2000792E252F0E947A2E242F0C947A2E0196FC
:105D3000272F0E947A2E0C94792EDC01CB01FC01D6
:105D4000F999FECF06C0F2BDE1BDF89A319600B4D4
:0E5D50000D9241505040B8F70895F894FFCFDF
:105D5E00C800C501010102000400040401191A1B48
:105D6E001C1D1E1F202122CB26D02611271227CE26
:105D7E0026CF2601659200010202020206060609DE
:105D8E0009090909090F0F0F0F0F0F15151518190E
:105D9E001919191919191919192324403B22F80C2C
:0A5DAE00BD0C9B0C400C590C720C4C
:00000001FF
